:100000000C942A001895000018950000189500001F
:10001000189500001895000018950000189500002C
:10002000189500001895000018950000189500001C
:10003000189500001895000018950000189500000C
:1000400018950000189500001895000018950000FC
:10005000189500008FE58DBFC0E4E0E44E2E84E0EB
:100060008EBFD4E0F4E05F2EEEEFF3E0A0E6B0E068
:1000700088278D933197E9F783E389B980E080BDC4
:1000800088E18AB9662480EE81BB80E082BB0027CC
:10009000BB27A0E38C9182FB0EF401E041E0041742
:1000A00011F00C946200BB27A2E38C9185FB88279A
:1000B00080F9809580FBBB27A2E38C9185F98C9316
:1000C0008299FECF0027BB27A0E38C9183FB0EF41F
:1000D00001E041E0041711F00C947D00BB27A2E37E
:1000E0008C9186FB882780F9809580FBBB27A2E353
:1000F0008C9186F98C938399FECF0027BB27A0E3D0
:100100008C9184FB0EF401E041E0041711F00C9493
:100110008F000E9491000E9498008499FECF0C9459
:100120004700979A84EF91E00E94B600979808954F
:10013000E2E9F1E00E949F000E94A60008950E945B
:10014000C500802D11F005D0FACF08958DE001D0C3
:100150008AE05D9BFECF8CB908953197F1F7089541
:10016000689462F80895E89462F80895EF93FF9315
:10017000EE27E82BE92B31F0E0EDF7E03197F1F7CE
:100180000197D1F7FF91EF910895C895319600201E
:10019000089541746D656C2D4576616C7561746967
:0A01A0006F6E2D426F617264000063
:00000001FF
